:100000000C9453020C947F1F0C94AC1F0C947B0235
:100010000C947B020C947B020C947B020C947B026C
:100020000C947B020C947B020C947B020C947B025C
:100030000C947B020C947B020C947B020C947B024C
:100040000C94D91F0C947B020C949C210C94EE21EF
:100050000C947B020C947B020C947B020C947B022C
:100060000C947B020C947B02000021104220633030
:100070008440A550C660E770088129914AA16BB100
:100080008CC1ADD1CEE1EFF13112100273325222A8
:10009000B5529442F772D662399318837BB35AA350
:1000A000BDD39CC3FFF3DEE3622443342004011478
:1000B000E664C774A44485546AA54BB528850995A0
:1000C000EEE5CFF5ACC58DD5533672261116300648
:1000D000D776F6669556B4465BB77AA719973887F0
:1000E000DFF7FEE79DD7BCC7C448E5588668A77808
:1000F0004008611802282338CCC9EDD98EE9AFF940
:10010000488969990AA92BB9F55AD44AB77A966AE7
:10011000711A500A333A122AFDDBDCCBBFFB9EEB8F
:10012000799B588B3BBB1AABA66C877CE44CC55CB7
:10013000222C033C600C411CAEED8FFDECCDCDDDDF
:100140002AAD0BBD688D499D977EB66ED55EF44E87
:10015000133E322E511E700E9FFFBEEFDDDFFCCF2F
:100160001BBF3AAF599F788F8891A981CAB1EBA183
:100170000CD12DC14EF16FE18010A100C230E320FF
:100180000450254046706760B9839893FBA3DAB3A7
:100190003DC31CD37FE35EF3B1029012F322D2324F
:1001A0003542145277625672EAB5CBA5A895898577
:1001B0006EF54FE52CD50DC5E234C324A01481049F
:1001C0006674476424540544DBA7FAB79987B89747
:1001D0005FE77EF71DC73CD7D326F2369106B016EF
:1001E00057667676154634564CD96DC90EF92FE907
:1001F000C899E9898AB9ABA944586548067827683F
:10020000C018E1088238A3287DCB5CDB3FEB1EFBE6
:10021000F98BD89BBBAB9ABB754A545A376A167A8E
:10022000F10AD01AB32A923A2EFD0FED6CDD4DCDB6
:10023000AABD8BADE89DC98D267C076C645C454CDE
:10024000A23C832CE01CC10C1FEF3EFF5DCF7CDF86
:100250009BAFBABFD98FF89F176E367E554E745E2E
:10026000932EB23ED10EF01E000000000000005F91
:1002700000000007000700147F147F14242A7F2A3F
:100280001223130864623649562050000807030001
:10029000001C2241000041221C002A1C7F1C2A084D
:1002A000083E0808008070300008080808080000B0
:1002B00060600020100804023E5149453E00427F24
:1002C000400072494949462141494D331814127F73
:1002D0001027454545393C4A494931412111090713
:1002E0003649494936464949291E00001400000094
:1002F0004034000000081422411414141414004166
:1003000022140802015909063E415D594E7C121122
:10031000127C7F494949363E414141227F4141415A
:100320003E7F494949417F090909013E41415173D5
:100330007F0808087F00417F41002040413F017F46
:10034000081422417F404040407F021C027F7F040E
:1003500008107F3E4141413E7F090909063E415157
:10036000215E7F09192946264949493203017F0147
:10037000033F4040403F1F2040201F3F4038403F48
:10038000631408146303047804036159494D43005E
:100390007F4141410204081020004141417F040295
:1003A000010204404040404000030708002054542C
:1003B00078407F284444383844444428384444280A
:1003C0007F385454541800087E090218A4A49C785D
:1003D0007F0804047800447D40002040403D007FB9
:1003E0001028440000417F40007C047804787C0899
:1003F0000404783844444438FC182424181824246D
:1004000018FC7C08040408485454542404043F4451
:10041000243C4040207C1C2040201C3C4030403C80
:1004200044281028444C9090907C4464544C4400E0
:100430000836410000007700000041360800020144
:100440000204023C2623263C000000002400270072
:100450002A0000000000250028002B0000000000FA
:1004600023002600290004040404040404040202F6
:100470000202020203030303030301020408102023
:10048000408001020408102001020408102000002E
:100490000007000201000003040600000000000045
:1004A000000082085D2311241FBECFEFD8E0DEBF1D
:1004B000CDBF11E0A0E0B1E0E4E4F8E502C00590B2
:1004C0000D92AE37B107D9F717E0AEE7B1E001C042
:1004D0001D92A338B107E1F714E0C6EAD4E004C0E6
:1004E0002297FE010E941C2CC23AD107C9F70E9434
:1004F000B4230C94202C0C940000FB01DC0102C0FE
:1005000001900D9241505040D8F70895FB01DC0155
:1005100001900D920020E1F7089561E070E040E065
:1005200050E016C0342F2227FB01E453FA4F80819C
:10053000E82FF0E0852F9927E827F927EE0FFF1F16
:10054000E859FF4F45915491422753276F5F7F4FE2
:100550008091040690910506861797071CF7409333
:100560001C0650931D06E0910406F0910506E25327
:10057000FA4F4083E0910406F0910506E353FA4FE9
:10058000508380910406909105060296909305068B
:10059000809304060895AF92BF92CF92DF92EF92BC
:1005A000FF920F931F93CF93DF93109261051092E8
:1005B00060058FEF809364051092630510926205C9
:1005C0008AEE80939A0186EA80939B0110929C01A7
:1005D00084E090E09093F1048093F00483E090E055
:1005E0009093F3048093F20440E050E0C1E0D0E047
:1005F00031E0E32EF12C012D112D109263051092A4
:100600006205BE01042E02C0660F771F0A94E2F74E
:1006100066C08091620590916305FC01EE0FFF1F9B
:10062000E80FF91FE45FFA4F808190E0862397235B
:10063000892BB9F0E091F204F091F304E756FE4FF4
:1006400020818091F0049091F1045701680104C069
:10065000AA0CBB1CCC1CDD1C8A95D2F72A2920834E
:1006600019C0E091F204F091F304E756FE4F2081A7
:100670008091F0049091F1045701680104C0AA0C24
:10068000BB1CCC1CDD1C8A95D2F7D601C501809518
:10069000822380838091F0049091F10401969093DD
:1006A000F1048093F0048091F0049091F104089794
:1006B0006CF01092F1041092F0048091F204909189
:1006C000F30401969093F3048093F2048091620501
:1006D00090916305019690936305809362058091E4
:1006E0006205909163054C970CF493CF4F5F5F4F79
:1006F0004830510509F081CF40E050E0C1E0D0E042
:10070000B1E0EB2EF12C012D112D1092630510920A
:100710006205BE01042E02C0660F771F0A94E2F73D
:1007200066C08091620590916305FC01EE0FFF1F8A
:10073000E80FF91FE45FFA4F818190E08623972349
:10074000892BB9F0E091F204F091F304E756FE4FE3
:1007500020818091F0049091F1045701680104C058
:10076000AA0CBB1CCC1CDD1C8A95D2F72A2920833D
:1007700019C0E091F204F091F304E756FE4F208196
:100780008091F0049091F1045701680104C0AA0C13
:10079000BB1CCC1CDD1C8A95D2F7D601C501809507
:1007A000822380838091F0049091F10401969093CC
:1007B000F1048093F0048091F0049091F104089783
:1007C0006CF01092F1041092F0048091F204909178
:1007D000F30401969093F3048093F20480916205F0
:1007E00090916305019690936305809362058091D3
:1007F0006205909163054C970CF493CF4F5F5F4F68
:100800004430510509F081CF44E050E0C1E0D0E030
:1008100031E0E32EF12C012D112D10926305109281
:100820006205BE01042E02C0660F771F0A94E2F72C
:1008300066C08091620590916305FC01EE0FFF1F79
:10084000E80FF91FE45FFA4F818190E08623972338
:10085000892BB9F0E091F204F091F304E756FE4FD2
:1008600020818091F0049091F1045701680104C047
:10087000AA0CBB1CCC1CDD1C8A95D2F72A2920832C
:1008800019C0E091F204F091F304E756FE4F208185
:100890008091F0049091F1045701680104C0AA0C02
:1008A000BB1CCC1CDD1C8A95D2F7D601C5018095F6
:1008B000822380838091F0049091F10401969093BB
:1008C000F1048093F0048091F0049091F104089772
:1008D0006CF01092F1041092F0048091F204909167
:1008E000F30401969093F3048093F20480916205DF
:1008F00090916305019690936305809362058091C2
:100900006205909163054B970CF493CF4F5F5F4F57
:100910004830510509F081CF40E050E0C1E0D0E01F
:10092000B1E0EB2EF12C012D112D109263051092E8
:100930006205BE01042E02C0660F771F0A94E2F71B
:1009400066C08091620590916305FC01EE0FFF1F68
:10095000E80FF91FE45FFA4F828190E08623972326
:10096000892BB9F0E091F204F091F304E756FE4FC1
:1009700020818091F0049091F1045701680104C036
:10098000AA0CBB1CCC1CDD1C8A95D2F72A2920831B
:1009900019C0E091F204F091F304E756FE4F208174
:1009A0008091F0049091F1045701680104C0AA0CF1
:1009B000BB1CCC1CDD1C8A95D2F7D601C5018095E5
:1009C000822380838091F0049091F10401969093AA
:1009D000F1048093F0048091F0049091F104089761
:1009E0006CF01092F1041092F0048091F204909156
:1009F000F30401969093F3048093F20480916205CE
:100A000090916305019690936305809362058091B0
:100A10006205909163054B970CF493CF4F5F5F4F46
:100A20004830510509F081CF84E090E09093F104C3
:100A30008093F00483E090E09093F3048093F204B9
:100A400081E090E0909363058093620541E0E42E9D
:100A5000F12C012D112D8EC080916405880F80939B
:100A60006405809164052091640590E034E09595DB
:100A700087953A95E1F781709070221F2227221FF7
:100A800030E08217930721F080916405816003C0F4
:100A9000809164058E7F8093640520916405E091C8
:100AA000F204F091F304E756FE4F80814091F00488
:100AB0005091F10490E002C0959587954A95E2F730
:100AC00030E08227932780FF17C0E091F204F09175
:100AD000F304E756FE4F20818091F0049091F104D9
:100AE000B801A70104C0440F551F661F771F8A95E0
:100AF000D2F7242B208319C0E091F204F091F30483
:100B0000E756FE4F20818091F0049091F104570147
:100B1000680104C0AA0CBB1CCC1CDD1C8A95D2F752
:100B2000D601C5018095822380838091F004909145
:100B3000F10401969093F1048093F0048091F00405
:100B40009091F10408976CF01092F1041092F00467
:100B50008091F2049091F30401969093F3048093B2
:100B6000F20480916205909163050196909363056C
:100B7000809362058091620590916305855992404A
:100B80000CF46ACFDF91CF911F910F91FF90EF90FE
:100B9000DF90CF90BF90AF90089540916405209171
:100BA00064058091640530E03595279550E0422733
:100BB00053274170507090E095958795959587954E
:100BC000817090704817590709F180916105209153
:100BD000600590E0FC01EE0FFF1FE80FF91FE20F28
:100BE000F11DE45FFA4F4081209162053091630569
:100BF00081E090E0A0E0B0E004C0880F991FAA1F38
:100C0000BB1F2A95D2F7482B408321C080916105F4
:100C10002091600590E0FC01EE0FFF1FE80FF91F27
:100C2000E20FF11DE45FFA4F40812091620530919F
:100C3000630581E090E0A0E0B0E004C0880F991F58
:100C4000AA1FBB1F2A95D2F78095842380838091A9
:100C50006205909163050196909363058093620508
:100C6000209164058091640590E095958795959510
:100C7000879530E08227932780FF21C0809161050E
:100C80002091600590E0FC01EE0FFF1FE80FF91FB7
:100C9000E20FF11DE45FFA4F40812091620530912F
:100CA000630581E090E0A0E0B0E004C0880F991FE8
:100CB000AA1FBB1F2A95D2F7482B408321C08091E1
:100CC00061052091600590E0FC01EE0FFF1FE80F29
:100CD000F91FE20FF11DE45FFA4F40812091620598
:100CE0003091630581E090E0A0E0B0E004C0880F9F
:100CF000991FAA1FBB1F2A95D2F780958423808352
:100D000080916205909163050196909363058093AD
:100D100062050895CF93DF931092610510926005EC
:100D200010926405109263051092620581E090E0D4
:100D300045C0C0E0D0E080916405880F80936405D1
:100D4000E0919005F0919105EB59FA4F808190E088
:100D50000C2E02C0959587950A94E2F780FF04C097
:100D600080916405816003C0809164058E7F8093CB
:100D700064050E94CD0580916205909163050897F6
:100D8000A4F01092630510926205809160058F5F58
:100D90008093600580916005833038F01092600583
:100DA000809161058F5F809361052196C830D105E0
:100DB00011F680919005909191050196909391057F
:100DC0008093900580919005909191058A970CF4FD
:100DD000B0CF80916405880F80936405809164058D
:100DE0008E7F809364050E94CD0580916405880FF5
:100DF00080936405809164058E7F809364050E94D2
:100E0000CD05DF91CF9108958091640583FFC6C021
:100E10008091640586FFC2C004C08091640586FD90
:100E2000C1C080916405880F80936405809164053A
:100E30008E7F809364058091FE0480FFBCC080910A
:100E4000640580FFB8C004C08091640580FDB7C010
:100E5000809161052091600590E0FC01EE0FFF1F7D
:100E6000E80FF91FE20FF11DE45FFA4F4081209176
:100E700062053091630581E090E0A0E0B0E004C03D
:100E8000880F991FAA1FBB1F2A95D2F7809584232C
:100E90008083809161058F5F8093610580916005FB
:100EA000882301F5809161058C31E0F01092610595
:100EB00080916205909163050197909363058093FB
:100EC0006205809162059091630597FF0BC087E0F2
:100ED00090E09093630580936205809160058F5F39
:100EE0008093600580916005813079F4809161057F
:100EF0008C3158F0109261058091620590916305E4
:100F0000019790936305809362058091600581301D
:100F1000A9F4809161058B3189F4809162059091EB
:100F2000630504975CF410926105809162059091CD
:100F30006305019790936305809362058091620534
:100F40009091630597FF0BC087E090E09093630555
:100F500080936205809160058F5F8093600580912A
:100F60006005823009F04CC0809161058B3108F436
:100F700047C01092610580916205909163050197C9
:100F8000909363058093620580916205909163055B
:100F900097FF36C083E08093090608958091640529
:100FA00083FF3BCF80916405880F80936405809117
:100FB000640581603ECF8091FE0480FF45CF809123
:100FC00061052091600590E0FC01EE0FFF1FE80F26
:100FD000F91FE20FF11DE45FFA4F40812091620595
:100FE0003091630581E090E0A0E0B0E004C0880F9C
:100FF000991FAA1FBB1F2A95D2F7482B408349CFC0
:1010000008958091640587FF19C08091640582FF6F
:1010100015C004C08091640582FD14C080916405F0
:101020008E7F8093640580918F0590E095958795DC
:1010300080938F0580918F058F7713C08091640511
:1010400087FFE8CF8091640581608093640580917B
:101050008F0590E09595879580938F0580918F05FA
:10106000806880938F0580916405880F8093640564
:10107000089580910B058F5F80930B0580910B0580
:10108000883000F110920B05E0915C01F0915D0158
:10109000E756FE4F80818093F40480915C0190912B
:1010A0005D01019790935D0180935C0180915C01EB
:1010B00090915D01892B31F48CE291E090935D0178
:1010C00080935C01E6E1F0E0DF01AC50BB4F8C9116
:1010D00090E0959587958C939F0121503040F901C0
:1010E000EC50FB4F808180FF03C08C91806802C070
:1010F0008C918F778C938FEF2F3F380711F0F90188
:10110000E3CF0895109281011092800189E691E069
:1011100090937F0180937E018FE0809386018EE023
:101120008093870181E18093880180E18093890128
:1011300082E180938A0108954F925F926F927F922D
:101140008F929F92AF92BF92CF92DF92EF92FF92D7
:101150000F931F93DF93CF93CDB7DEB7C854D04022
:101160000FB6F894DEBF0FBECDBF20E030E00FE138
:10117000402E512C4C0E5D1E18E2C12ED12CCC0EEF
:10118000DD1E8E010F5C1F4FBAE3EB2EF12CEC0E2F
:10119000FD1EF901E759FA4F8081F201E20FF31FBA
:1011A0008083F901EF58FA4F8081F601E20FF31FB7
:1011B0008083F901E758FA4F8081F801E20FF31FAD
:1011C0008083F901EF57FA4F8081F701E20FF31F97
:1011D00080832F5F3F4F28303105D9F68FE2FE0123
:1011E000EE5BFF4F808380918905FE01ED5BFF4F31
:1011F000808380918A05FE01EC5BFF4F80838091A4
:101200008B05FE01EB5BFF4F808380918C05FE0117
:10121000EA5BFF4F80831FA218AA19AEFE01E95BAB
:10122000FF4F108289A980933F068AA980934006C8
:101230008BA9809341068CA9809342068DA9809347
:1012400043068EA9809344068FA98093450688ADF6
:10125000809346061092470681E080938401809334
:1012600085018EE791E063E040E00E94C11B8EE7BC
:1012700091E060E071E00E94FD1D8EE791E063E087
:1012800047E30E94C11B8EE791E0B8010E94D02481
:101290008EE791E065E040E00E94C11B8EE791E09F
:1012A0006AE071E00E94FD1D8EE791E065E042E397
:1012B0000E94C11B8EE791E0B7010E94D0248EE707
:1012C00091E067E040E00E94C11B8EE791E064E19D
:1012D00071E00E94FD1D8EE791E067E047E30E9408
:1012E000C11B4E010894811C911CC401B6010E94CF
:1012F0008226A7E0AA2EB12CAC0EBD1EC501B401FA
:1013000040E050E028E030E00E94B426FDE0CF2E1F
:10131000D12CCC0EDD1EC601B5010E941227C601DC
:101320006EE171E00E942F263C01E3E1EE2EF12CEC
:10133000EC0EFD1EC701B2010E9482268E01075EDF
:101340001F4FC801B70147E050E028E030E00E949D
:10135000B426C301B8010E944B26BC018EE791E080
:101360000E94EF23C8010E941C27C7010E941C276E
:10137000C6010E942227C5010E941C27C4010E94A9
:101380001C27C85BDF4F0FB6F894DEBF0FBECDBF82
:10139000CF91DF911F910F91FF90EF90DF90CF9051
:1013A000BF90AF909F908F907F906F905F904F9085
:1013B00008954F925F926F927F928F929F92AF9219
:1013C000BF92CF92DF92EF92FF920F931F93DF9322
:1013D000CF93CDB7DEB7C854D0400FB6F894DEBF78
:1013E0000FBECDBF20E030E06FE1462E512C4C0EF9
:1013F0005D1E58E2C52ED12CCC0EDD1E8E010F5C79
:101400001F4F4AE3E42EF12CEC0EFD1EF901E859C2
:10141000FA4F8081F201E20FF31F8083F901E05956
:10142000FA4F8081F601E20FF31F8083F901E8583B
:10143000FA4F8081F801E20FF31F8083F901E05831
:10144000FA4F8081F701E20FF31F80832F5F3F4F38
:1014500028303105D9F68FE2FE01EE5BFF4F808325
:1014600080918805FE01ED5BFF4F808380918905A7
:10147000FE01EC5BFF4F808380918A05FE01EB5BF0
:10148000FF4F808380918B05FE01EA5BFF4F8083D5
:101490001FA218AA19AEFE01E95BFF4F108289A9AD
:1014A00080933F068AA9809340068BA980934106CA
:1014B0008CA9809342068DA9809343068EA98093C0
:1014C00044068FA98093450688AD80934606109206
:1014D000470681E080938401809385018EE791E047
:1014E00063E040E00E94C11B8EE791E060E071E0A4
:1014F0000E94FD1D8EE791E063E047E30E94C11B5F
:101500008EE791E0B8010E94D0248EE791E065E07B
:1015100040E00E94C11B8EE791E06AE071E00E940A
:10152000FD1D8EE791E065E042E30E94C11B8EE75E
:1015300091E0B7010E94D0248EE791E067E040E09F
:101540000E94C11B8EE791E064E171E00E94FD1DE5
:101550008EE791E067E047E30E94C11B4E010894CB
:10156000811C911CC401B6010E94822627E0A22E94
:10157000B12CAC0EBD1EC501B40140E050E028E026
:1015800030E00E94B4269DE0C92ED12CCC0EDD1E89
:10159000C601B5010E941227C6016EE171E00E94EA
:1015A0002F263C0183E1E82EF12CEC0EFD1EC70135
:1015B000B2010E9482268E01075E1F4FC801B7014B
:1015C00047E050E028E030E00E94B426C301B801B3
:1015D0000E944B26BC018EE791E00E94EF23C801D8
:1015E0000E941C27C7010E941C27C6010E942227B7
:1015F000C5010E941C27C4010E941C27C85BDF4F45
:101600000FB6F894DEBF0FBECDBFCF91DF911F9113
:101610000F91FF90EF90DF90CF90BF90AF909F9091
:101620008F907F906F905F904F900895EF92FF9210
:101630000F931F93609126067091270680912806CC
:101640009091290664527C4B814090400E94422A2E
:1016500028EA3DEF40EE5AE40E94A72960932A064B
:1016600070932B0680932C0690932D0660912A068A
:1016700070912B0680912C0690912D060E947D2A58
:101680000E94142A60932E06E0902A06F0902B0602
:1016900000912C0610912D0660912E0670E088278F
:1016A00077FD8095982F0E94422A9B01AC01C801CA
:1016B000B7010E943E2920E030E040E057E40E945C
:1016C0004B2B60932A0670932B0680932C069093E5
:1016D0002D0660912A0670912B0680912C06909120
:1016E0002D0620E030E040E05FE30E943F290E94A9
:1016F0007D2A0E94142A7093300660932F0683E09F
:1017000090E0A0E0B0E08093310690933206A09381
:101710003306B09334068091310690913206A09141
:101720003306B0913406BA2FA92F982F88278093BB
:10173000310690933206A0933306B093340620917D
:101740003106309132064091330650913406809133
:101750002E0690E0A0E0B0E0822B932BA42BB52BBB
:101760008093310690933206A0933306B0933406EB
:101770008091310690913206A0913306B0913406E3
:101780000FE0880F991FAA1FBB1F0A95D1F78093FE
:10179000310690933206A0933306B093340620911D
:1017A00031063091320640913306509134068091D3
:1017B0002F0690913006A0E0B0E0822B932BA42B53
:1017C000B52B8093310690933206A0933306B093E5
:1017D00034068091310690913206A0913306B09183
:1017E000340614E0880F991FAA1FBB1F1A95D1F762
:1017F0008093310690933206A0933306B09334065B
:1018000060912606709127068091280690912906FE
:1018100064587543804090400E94422A28EA3DEF78
:1018200040EE5AE40E94A72960932A0670932B0683
:1018300080932C0690932D0660912A0670912B06BA
:1018400080912C0690912D060E947D2A0E94142AD8
:1018500060932E06E0902A06F0902B0600912C064D
:1018600010912D0660912E0670E0882777FD8095F7
:10187000982F0E94422A9B01AC01C801B7010E9427
:101880003E2920E030E040E057E40E944B2B60937B
:101890002A0670932B0680932C0690932D06609158
:1018A0002A0670912B0680912C0690912D0620E03F
:1018B00030E040E05FE30E943F290E947D2A0E94C1
:1018C000142A7093300660932F0682E090E0A0E027
:1018D000B0E08093350690933606A0933706B09318
:1018E00038068091350690913606A0913706B09162
:1018F0003806BA2FA92F982F882780933506909302
:101900003606A0933706B0933806209135063091FD
:101910003606409137065091380680912E0690E0A9
:10192000A0E0B0E0822B932BA42BB52B809335063F
:1019300090933606A0933706B0933806809135060B
:1019400090913606A0913706B0913806EFE0880FE7
:10195000991FAA1FBB1FEA95D1F780933506909374
:101960003606A0933706B09338062091350630919D
:101970003606409137065091380680912F06909197
:101980003006A0E0B0E0822B932BA42BB52B8093E4
:10199000350690933606A0933706B09338068091AB
:1019A000350690913606A0913706B091380674E05E
:1019B000880F991FAA1FBB1F7A95D1F78093350610
:1019C00090933606A0933706B09338061F910F9177
:1019D000FF90EF900895EF92FF920F931F938091E5
:1019E000990590E090933A068093390680913906E4
:1019F00090913A06A0E0B0E08093260690932706E7
:101A0000A0932806B093290680919A0590E09093C0
:101A10003A06809339062091260630912706409198
:101A20002806509129068091390690913A06982F00
:101A30008827A0E0B0E0820F931FA41FB51F8093FA
:101A4000260690932706A0932806B0932906809136
:101A50009B0590E090933A068093390620912606E4
:101A60003091270640912806509129068091390629
:101A700090913A06A0E0B0E0DC0199278827820F18
:101A8000931FA41FB51F8093260690932706A0934B
:101A90002806B093290680919C0590E090933A0621
:101AA000809339062091260630912706409128061A
:101AB000509129068091390690913A06A0E0B0E055
:101AC000B82FAA2799278827820F931FA41FB51F15
:101AD0008093260690932706A0932806B0932906A4
:101AE000609126067091270680912806909129061C
:101AF00064527C4B814090400E94422A28EA3DEF8C
:101B000040EE5AE40E94A72960932A0670932B06A0
:101B100080932C0690932D0660912A0670912B06D7
:101B200080912C0690912D060E947D2A0E94142AF5
:101B300060932E06E0902A06F0902B0600912C066A
:101B400010912D0660912E0670E0882777FD809514
:101B5000982F0E94422A9B01AC01C801B7010E9444
:101B60003E2920E030E040E057E40E944B2B609398
:101B70002A0670932B0680932C0690932D06609175
:101B80002A0670912B0680912C0690912D0620E05C
:101B900030E040E05FE30E943F290E947D2A0E94DE
:101BA000142A7093300660932F0683E090E0A0E043
:101BB000B0E08093310690933206A0933306B09341
:101BC00034068091310690913206A0913306B0918F
:101BD0003406BA2FA92F982F882780933106909327
:101BE0003206A0933306B09334062091310630912B
:101BF0003206409133065091340680912E0690E0D3
:101C0000A0E0B0E0822B932BA42BB52B8093310660
:101C100090933206A0933306B09334068091310638
:101C200090913206A0913306B09134067FE0880F80
:101C3000991FAA1FBB1F7A95D1F780933106909305
:101C40003206A0933306B0933406209131063091CA
:101C50003206409133065091340680912F069091C0
:101C60003006A0E0B0E0822B932BA42BB52B809301
:101C7000310690933206A0933306B09334068091D8
:101C8000310690913206A0913306B091340664E09B
:101C9000880F991FAA1FBB1F6A95D1F78093310641
:101CA00090933206A0933306B093340660912606D3
:101CB00070912706809128069091290664587543F3
:101CC000804090400E94422A28EA3DEF40EE5AE4CC
:101CD0000E94A72960932A0670932B0680932C06F6
:101CE00090932D0660912A0670912B0680912C0608
:101CF00090912D060E947D2A0E94142A60932E0640
:101D0000E0902A06F0902B0600912C0610912D06EB
:101D100060912E0670E0882777FD8095982F0E94AD
:101D2000422A9B01AC01C801B7010E943E2920E074
:101D300030E040E057E40E944B2B60932A067093FA
:101D40002B0680932C0690932D0660912A067091A5
:101D50002B0680912C0690912D0620E030E040E08B
:101D60005FE30E943F290E947D2A0E94142A7093FB
:101D7000300660932F0682E090E0A0E0B0E0809310
:101D8000350690933606A0933706B09338068091B7
:101D9000350690913606A0913706B0913806BA2FD5
:101DA000A92F982F88278093350690933606A09305
:101DB0003706B093380620913506309136064091AB
:101DC00037065091380680912E0690E0A0E0B0E0F2
:101DD000822B932BA42BB52B80933506909336063C
:101DE000A0933706B0933806809135069091360659
:101DF000A0913706B09138064FE0880F991FAA1FAF
:101E0000BB1F4A95D1F78093350690933606A09371
:101E10003706B0933806209135063091360640914A
:101E200037065091380680912F0690913006A0E039
:101E3000B0E0822B932BA42BB52B80933506909387
:101E40003606A0933706B0933806809135069091F8
:101E50003606A0913706B091380634E0880F991FF6
:101E6000AA1FBB1F3A95D1F780933506909336068B
:101E7000A0933706B09338061F910F91FF90EF9013
:101E8000089580911E0690911F06019690931F065B
:101E900080931E0685E00E944821892B21F08091C5
:101EA0009701806803C0809197018F778093970195
:101EB000809198018F5F809398018091980188307C
:101EC00009F5E0915A01F0915B0180919701E75685
:101ED000FE4F808380915A0190915B01019790930E
:101EE0005B0180935A0180915A0190915B01892B8B
:101EF00031F48CE291E090935B0180935A0110924F
:101F0000980107C08091970190E0959587958093FF
:101F1000970181E080930B06089580911E069091B1
:101F20001F06019690931F0680931E06809113064C
:101F30009091140601979093140680931306809154
:101F40000C06843021F080910C06853009F5109242
:101F50001A061092190680911B06815080931B0669
:101F600086E00E944821019719F486E060E002C0F3
:101F700086E061E00E94F42080910C06853041F4F7
:101F800086E00E944821019719F486E080930C06B0
:101F900080910C06873029F080910C06883009F07A
:101FA00070C08091190690911A06019690931A06B6
:101FB000809319068091190690911A068036910532
:101FC0005CF010921A0610921906809118068F5F25
:101FD0008093180680911806E091EE04F091EF04CA
:101FE000E756FE4F80812091F0043091F10490E09B
:101FF00002C0959587952A95E2F780FF03C086E099
:1020000061E002C086E060E00E94F4208091F0046C
:102010009091F10401969093F1048093F0048091E3
:10202000F0049091F1040897D1F41092F104109209
:10203000F0048091EE049091EF0401969093EF04E8
:102040008093EE048091EE049091EF0483559340C9
:1020500034F081E090E09093EF048093EE0480915F
:102060000C06883071F42091EC043091ED048091DD
:10207000EE049091EF042817390719F489E0809352
:102080000C0681E080930E0683E060E00E94F4205D
:1020900008958FE190E029C080912006909121065B
:1020A000A0912206B09123062091240630912506A6
:1020B00004C0B595A795979587952A95D2F780FF87
:1020C00003C08AE061E002C08AE060E00E94F42080
:1020D00087E061E00E94F42087E060E00E94F42045
:1020E0008091240690912506019790932506809370
:1020F0002406809124069091250697FFCDCF8CE091
:1021000061E00E94F4208CE060E00E94F4208AE00C
:1021100060E00E94F420089585EF94E2A0E0B0E032
:102120008093200690932106A0932206B093230665
:102130000E94491082E990EDA5E6B1E08093200667
:1021400090932106A0932206B09323060E94491083
:1021500083E990ECACE4BAE28093200690932106E8
:10216000A0932206B09323060E94491084E194ECC8
:10217000A5E4B0E48093200690932106A093220664
:10218000B09323060E944910809131069091320647
:10219000A0913306B09134068093200690932106D7
:1021A000A0932206B09323060E944910089582E965
:1021B00090EDA5E7B0E08093200690932106A093D0
:1021C0002206B09323060E94491080913506909113
:1021D0003606A0913706B09138068093200690937A
:1021E0002106A0932206B09323060E944910089569
:1021F00081E190E5A7E5B0E0809320069093210669
:10220000A0932206B09323060E94491083E990EC24
:10221000ACE4BAE28093200690932106A0932206B4
:10222000B09323060E9449108091310690913206A6
:10223000A0913306B0913406809320069093210636
:10224000A0932206B09323060E94491085EF94E2E2
:10225000A0E0B0E08093200690932106A093220690
:10226000B09323060E94491084E194ECA5E4B0E405
:102270008093200690932106A0932206B093230614
:102280000E94491082E990EDA5E6B1E08093200616
:1022900090932106A0932206B09323060E94491032
:1022A0008FE090E0AEE0B0E08093200690932106AE
:1022B000A0932206B09323060E94491086E09EE078
:1022C000A7E0B5E08093200690932106A093220614
:1022D000B09323060E94491089EE91E3A2E0B0E09A
:1022E0008093200690932106A0932206B0932306A4
:1022F0000E9449108AE397E4A6E9B2E3809320069E
:1023000090932106A0932206B09323060E944910C1
:102310008BE390E0A0E0B0E080932006909321064C
:10232000A0932206B09323060E9449108CE091E00E
:10233000A0E0B0E08093200690932106A0932206AF
:10234000B09323060E9449108DE090E0A0E0B0E039
:102350008093200690932106A0932206B093230633
:102360000E944910089580E48093990588E780933E
:102370009A0587EE80939B0589E180939C050E94D6
:10238000EB0C0E94F81080E00E946C1F80E061E47A
:102390007FE043E050E00E94491F089580E00E94E2
:1023A0006C1F80E061E47FE043E050E00E94491F41
:1023B00081E00E946C1F809116068E7F8093160626
:1023C000809116068D7F8093160688E060E00E945B
:1023D000F4208DE060E00E94F4200E948C108CE2DA
:1023E00091E090935B0180935A0110920B0510923B
:1023F000090610920606109207061092180610920F
:10240000170681E080930C0610920D0680930A0651
:102410000895CF93DF9380ED8093CD050E948D02C8
:10242000C1E0D0E009C0FE01E453FA4F60818DE5C0
:1024300097E00E941D232196809104069091050645
:102440008C179D0784F7DF91CF910895FF920F932A
:102450001F93809102058A3A09F050C080910105CE
:102460008A3A09F04BC0809100058E3609F046C0CB
:102470008091FF048A3009F041C082E08093090610
:10248000109260051092610587E090E090936305DB
:10249000809362058FEF8093640510920806809107
:1024A0005E018F5F80935E0133E0F32EF092CE05E4
:1024B0001092CF0585E18093D0051092D10510923E
:1024C000D20506E010E010930506009304060E9472
:1024D0000912F092CE051092CF0586E18093D005C7
:1024E00080915E018093D105809108068093D2058A
:1024F00010930506009304060E9409121F910F9184
:10250000FF90089510926105109260051092640585
:10251000109291051092900514C110928F05809130
:10252000610590E020916005FC01EE0FFF1FE80FB0
:10253000F91FE20FF11DE45FFA4F808186FF04C0AE
:1025400080916405806803C0809164058F778093D3
:1025500064050E9401088091610590E0209160056A
:10256000FC01EE0FFF1FE80FF91FE20FF11DE45F02
:10257000FA4F808184FF04C080916405806803C0A5
:10258000809164058F77809364050E940108809193
:10259000610590E020916005FC01EE0FFF1FE80F40
:1025A000F91FE20FF11DE45FFA4F808182FF04C042
:1025B00080916405806803C0809164058F77809363
:1025C00064050E9401088091610590E020916005FA
:1025D000FC01EE0FFF1FE80FF91FE20FF11DE45F92
:1025E000FA4F808180FF04C080916405806803C039
:1025F000809164058F77809364050E940108809123
:1026000060058F5F8093600580916005833038F0AE
:1026100010926005809161058F5F809361058091C4
:10262000610590E020916005FC01EE0FFF1FE80FAF
:10263000F91FE20FF11DE45FFA4F808186FF04C0AD
:1026400080916405806803C0809164058F778093D2
:1026500064050E9401088091610590E02091600569
:10266000FC01EE0FFF1FE80FF91FE20FF11DE45F01
:10267000FA4F808184FF04C080916405806803C0A4
:10268000809164058F77809364050E940108809192
:10269000610590E020916005FC01EE0FFF1FE80F3F
:1026A000F91FE20FF11DE45FFA4F808182FF04C041
:1026B00080916405806803C0809164058F77809362
:1026C00064050E9401088091610590E020916005F9
:1026D000FC01EE0FFF1FE80FF91FE20FF11DE45F91
:1026E000FA4F808180FF04C080916405806803C038
:1026F000809164058F77809364050E940108809122
:1027000060058F5F8093600580916005833038F0AD
:1027100010926005809161058F5F80936105E09163
:102720009005F091910580918F05EB59FA4F8083C8
:1027300080919005909191050196909391058093D9
:102740009005809190059091910589970CF4E5CEC4
:1027500084E0809309068FE28093CE051092CF0526
:1027600087E18093D00580915E018093D1058091AF
:1027700008068093D2051092D3051092D4051092CA
:1027800091051092900517C0A0919005B091910508
:10279000E0919005F0919105EB59FA4F8081AB5291
:1027A000BA4F8C93809190059091910501969093EA
:1027B000910580939005809190059091910589975E
:1027C0001CF30E94D90982E390E090930506809360
:1027D00004060E940912089580919505813109F03F
:1027E00040C08093CE051092CF0581E98093D0053B
:1027F0001092D10594E59093D20583E58093D3059B
:1028000080E58093D40588E38093D5058EE480939A
:10281000D6059093D70588E48093D80580E280930D
:10282000D9058093DA0584E48093DB0586E58093FF
:10283000DC058DE28093DD059093DE0582E58093D3
:10284000DF0588E58093E00584E190E0909305063C
:10285000809304060E94091281E080930C06809305
:102860000A06809195058231E1F485E08093CE05DA
:102870001092CF0582E98093D00583E18093D10542
:1028800089E08093D20580E18093D30581E0809335
:10289000D40588E090E090930506809304060E949A
:1028A0000912809195058431D9F580919605803C77
:1028B00091F48091980580930F06809199058093FB
:1028C000100680919A058093110680919B05809354
:1028D00012060E94B31180919605813C71F480E04C
:1028E0000E946C1F0E94EB0C80E061E47FE043E0FB
:1028F00050E00E94491F0E94F81082E08093CE05AC
:102900001092CF0584E98093D00586E08093D105AD
:1029100085E090E090930506809304060E940912DA
:10292000809195058031D1F4909193059230B1F466
:1029300080919605809315069093CE051092CF0551
:1029400080E98093D00586E08093D10585E090E012
:1029500090930506809304060E94091280919505C4
:10296000803169F580919305813049F588E0809345
:10297000CE051092CF0580E98093D00587E480933F
:10298000D105809116068093D20580910A06809326
:10299000D30585E18093D4058CEF8093D505809194
:1029A00017068093D605809118068093D7058BE093
:1029B00090E090930506809304060E94091280918E
:1029C0009505863139F486E060E00E94F42081E0CC
:1029D00080930D0680919505873161F5809196056C
:1029E00080935E01809197058093080621E030E096
:1029F000F901E756FA4F8081F901EB59FA4F8083CC
:102A00002F5F3F4F2A32310599F70E949C0886E5D7
:102A100090E09093ED048093EC0481E090E090933B
:102A2000EF048093EE040E948A060E94CB0282E0AB
:102A300080930D0680919505893109F03EC0109272
:102A40001F0610921E06809107068F5F809307066F
:102A500080910706853110F01092070628E030E0DB
:102A600041E050E0E091EC04F091ED04D901AE5664
:102A7000BA4F8C91E756FE4F80838091EC04909181
:102A8000ED0401969093ED048093EC048091EC04A6
:102A90009091ED048355934024F05093ED044093BE
:102AA000EC042F5F3F4F24313105E1F680910D0694
:102AB000823019F483E080930D06809195058A3168
:102AC00009F04DC18091EC049091ED040197909331
:102AD000ED048093EC048091EC049091ED04892B3B
:102AE00031F482E593E09093ED048093EC048091BF
:102AF000EC049091ED0401979093ED048093EC0425
:102B00008091EC049091ED04892B31F482E593E0FF
:102B10009093ED048093EC048091EC049091ED048B
:102B200001979093ED048093EC048091EC049091D4
:102B3000ED04892B31F482E593E09093ED048093CA
:102B4000EC04E091EC04F091ED04E756FE4F85E5CE
:102B500080838091EC049091ED0401969093ED04B4
:102B60008093EC048091EC049091ED0483559340A4
:102B700034F081E090E09093ED048093EC04E091D8
:102B8000EC04F091ED04E756FE4F85E580838091DB
:102B9000EC049091ED0401969093ED048093EC0485
:102BA0008091EC049091ED048355934034F081E0E2
:102BB00090E09093ED048093EC04E091EC04F091AC
:102BC000ED04E756FE4F85E580838091EC049091FB
:102BD000ED0401969093ED048093EC048091EC0455
:102BE0009091ED048355934034F081E090E0909310
:102BF000ED048093EC04E091EC04F091ED04E756D1
:102C0000FE4F85E580838091EC049091ED04019660
:102C10009093ED048093EC048091EC049091ED048A
:102C20008355934034F081E090E09093ED048093DD
:102C3000EC04E091EC04F091ED04E756FE4F88ECD3
:102C400080838091EC049091ED0401969093ED04C3
:102C50008093EC048091EC049091ED0483559340B3
:102C600034F081E090E09093ED048093EC04E091E7
:102C7000EC04F091ED04E756FE4F8AE780838091E3
:102C8000EC049091ED0401969093ED048093EC0494
:102C90008091EC049091ED048355934034F081E0F1
:102CA00090E09093ED048093EC04E091EC04F091BB
:102CB000ED04E756FE4F10828091EC049091ED04F4
:102CC00001969093ED048093EC048091EC04909134
:102CD000ED048355934034F081E090E09093ED044F
:102CE0008093EC04E091EC04F091ED04E756FE4F84
:102CF00010828091EC049091ED0401969093ED0484
:102D00008093EC048091EC049091ED048355934002
:102D100034F081E090E09093ED048093EC04E09136
:102D2000EC04F091ED04E756FE4F10828091EC0424
:102D30009091ED0401969093ED048093EC048091C2
:102D4000EC049091ED048355934034F081E090E0E1
:102D50009093ED048093EC0484E080930D068091C1
:102D600095058F31E1F590919605903CD1F486E080
:102D70008093CE051092CF058FE98093D005909374
:102D8000D1051092D2051092D3051092D40510925D
:102D9000D50589E090E090930506809304060E9493
:102DA000091290919605913CD1F486E08093CE056E
:102DB0001092CF058FE98093D0059093D1051092A2
:102DC000D2051092D3051092D4051092D50589E052
:102DD00090E090930506809304060E9409121092D9
:102DE0009205109293051092CB051092CA05089592
:102DF00083E18093CE051092CF0589E18093D005C1
:102E000080915E018093D105809108068093D20560
:102E100088EE8093D30583E08093D40525E130E0EC
:102E20004EE150E0FA01E21BF30BD901AC50BB4F6D
:102E30008C91E453FA4F8083215030402930310582
:102E400089F71092E1051092E20586E190E09093F7
:102E50000506809304060E940912089583E080937A
:102E6000CE051092CF058AE18093D00580915E0156
:102E70008093D105809108068093D20586E090E08A
:102E800090930506809304060E94091208950F93FB
:102E90001F93CF93DF9320913B0630913C064091E6
:102EA0003D0650913E068091260690912706A091FE
:102EB0002806B0912906281739074A075B0709F445
:102EC0004EC080E00E946C1F0E94160B0E94F810FA
:102ED00080E061E47FE043E050E00E94491F809180
:102EE000260690912706A0912806B0912906809386
:102EF0003B0690933C06A0933D06B0933E068EE7BA
:102F000091E060E045E00E94C11B82E08093840173
:102F100081E08093850160913B0670913C06809131
:102F20003D0690913E060E94422A20E034E244E7AA
:102F300059E40E94A729AB01BC018EE791E023E090
:102F400030E00E94B7258EE791E060E04AE50E94FC
:102F5000C11B8EE791E062E271E00E94FD1D8DE5EC
:102F600097E00E94B022181619060CF50091CA05C8
:102F70001091CB058DE597E00E94E4220E561A4F82
:102F8000F80180838091CA059091CB0501969093BA
:102F9000CB058093CA058091CA059091CB05C8974F
:102FA00034F087E390E09093CB058093CA0580913D
:102FB0009205803D21F01092CB051092CA058091B8
:102FC0009205803D99F48091CA059091CB050597B3
:102FD0006CF02091CA053091CB058091930590E06B
:102FE00004968217930714F40E94EC1380910E0646
:102FF000813009F045C02091EC043091ED048091BE
:10300000EE049091EF048217930784F48091EC040E
:103010009091ED042091EE043091EF04821B930B0C
:103020006CE070E00E94E52B609317062091EC04A1
:103030003091ED048091EE049091EF042817390748
:1030400094F48091EC049091ED042091EE04309181
:10305000EF048E5A9C4F821B930B6CE070E00E9431
:10306000E52B609317062091EC043091ED048091DC
:10307000EE049091EF042817390711F41092170607
:1030800080910C06882309F4ECC080910C068130F5
:1030900009F058C080910D06882309F453C08AEFC7
:1030A00090E090935D0180935C018CE291E09093BD
:1030B0005B0180935A0180E00E946C1F81E00E94B6
:1030C0006C1F809116068E7F8093160680911606DF
:1030D00082608093160688E061E00E94F4208DE013
:1030E00061E00E94F4200E94D71080E06DE87FE04C
:1030F00042E050E00E94491F8091110625E0829F26
:10310000C001112490931406809313064091130676
:10311000509114068091120690E02BEF34E0BC0130
:10312000629FC001639F900D729F900D1124840FC8
:10313000951F909314068093130682E080930C06EB
:1031400080930A0680910C06823049F48091130620
:1031500090911406059718F483E080930C069091E3
:103160000C06933061F480910D06823040F080E4CB
:1031700080931B0684E080930C0690930A0680914E
:103180000C06843039F480911B06823018F485E0F7
:1031900080930C0680910C06863031F487E0809392
:1031A0000C0685E080930A0680910C06873009F0B2
:1031B00045C080911E0690911F06815C924110F0DF
:1031C0000E94CE11809117068530D0F48091EE04D4
:1031D0009091EF04CC979093EF048093EE0480914C
:1031E000EE049091EF041816190654F08091EE0445
:1031F0009091EF048E5A9C4F9093EF048093EE04CD
:10320000809117068334D0F08091EC049091ED0406
:10321000CC979093ED048093EC048091EC04909112
:10322000ED041816190654F08091EC049091ED0409
:103230008E5A9C4F9093ED048093EC0490910C0671
:10324000973049F480910D06843029F488E080930A
:103250000C0690930A0680910C06893011F40E94A6
:10326000CE11809109068630C0F520915A01309127
:103270005B0180915C0190915D018217930794F44A
:1032800080915C0190915D0120915A0130915B0128
:10329000845D9E4F821B930B8B3F91051CF081E058
:1032A00080930B0620915C0130915D0180915A0161
:1032B00090915B018217930784F480915C01909157
:1032C0005D0120915A0130915B01821B930B8B3F72
:1032D00091051CF081E080930B0680910B068130F4
:1032E00009F04AC10E943908809109068823D9F45F
:1032F00090910B069130B9F4809102058A3A99F4C5
:10330000809101058A3A79F4809100058A3A59F44E
:103310008091FF048A3A39F4909309068091160649
:1033200081608093160680910906813031F4809186
:103330000B06813011F40E9426128091090682301A
:1033400061F480910B06813041F40E9404071092D1
:103350000C0683E061E00E94F4208091090683302E
:1033600031F480910B06813011F40E948212809119
:103370000906843039F480910B06813019F485E018
:1033800080930906809109068530D1F480910B065F
:103390008130B1F405C00E943908809106068F5F24
:1033A00080930606809106068131A8F386E080931B
:1033B00009061092060684E18093070610920B0618
:1033C00080910906863009F0D7C080910B068130C4
:1033D00009F0D2C0809106068F5F80930606809127
:1033E0000606823008F44FC080910606893108F045
:1033F0004AC020915C0130915D0180915A01909109
:103400005B0182179307CCF480915C0190915D0180
:1034100020915A0130915B01821B930B45976CF010
:10342000C1E0D0E00E943908809106068F5F80934A
:1034300006062196C132D105A9F720915C01309191
:103440005D0180915A0190915B0128173907DCF4E6
:1034500080915C0190915D0120915A0130915B0156
:10346000845D9E4F821B930B45976CF0C1E0D0E0CA
:103470000E943908809106068F5F80930606219688
:10348000C132D105A9F7809106068934E1F4809113
:1034900000058535C1F48091FF048535A1F4809144
:1034A000FE04853581F48091FD04853561F48091B9
:1034B000FC04883C41F48091FB048A3721F40E948B
:1034C000CE110E942E17809107068431A1F48091BD
:1034D0000606823480F08091FF04853561F4809186
:1034E000FE048D3241F48091FD04863121F4109266
:1034F0000B060E94390880910706843111F58091EE
:1035000006068934F1F4809100058535F1F5809146
:10351000FF048D32D1F58091FE048631B1F511C0E2
:103520008091FF048D3221F08091FE04863191F567
:1035300085E5809300058DE28093FF0486E180930A
:10354000FE0480910606893431F480910706809349
:1035500008060E94F81680910606803668F01092E0
:103560000606809107068F5F809307068091070605
:10357000853110F01092070610920B0610920E067D
:10358000DF91CF911F910F910895809100058535AE
:1035900039F6CECF0E94CE110E942E17D2CFEF92D5
:1035A000FF920F931F930EE711E0C8010E942C1E9B
:1035B000C8010E94E51BC80160E045E00E94C11BF4
:1035C00052E0F52EF0928401EE24E394E09285011E
:1035D000C80166E271E00E94FD1D83E080938401D2
:1035E000F0928501C80163E040E00E94C11BC80160
:1035F00062E371E00E94FD1DE0928401F09285017A
:10360000C80167E045E00E94C11BC8016AE371E0A0
:103610000E94FD1D68EE73E080E090E00E94212092
:10362000C8010E94E51B82E060E00E94B52087E0AF
:1036300061E00E94B52085E060E00E94B52086E050
:1036400061E00E94B5208AE061E00E94B5208CE034
:1036500061E00E94B52088E061E00E94B5208DE025
:1036600061E00E94B52083E061E00E94B52087E020
:1036700060E00E94F4208CE060E00E94F4208AE088
:1036800060E00E94F42088E060E00E94F4208DE079
:1036900061E00E94F4200DE517E0C80140E052EC23
:1036A00061E070E00E942922C8010E940D230E945F
:1036B000B3118DE061E00E94F4201F910F91FF9003
:1036C000EF900895DC015196ED91FC915297808125
:1036D00057969C915797892B80835396ED91FC9137
:1036E0005497908158968C91589780958923808320
:1036F0005196ED91FC915297908157968C915797E6
:1037000080958923808330E840E050E070E01F9688
:10371000ED91FC915097908156968C91569780959B
:1037200089238083832F90E0862397231D96ED9134
:10373000FC911E9755962C915597892B21F08081ED
:10374000822B808304C080812095282320831F96AC
:10375000ED91FC915097808156969C915697892BBC
:10376000808336954F5F5F4F4830510581F6519603
:10377000ED91FC915297808157969C91892B808383
:1037800008950F931F93CF93DF93EC01142F062F0F
:10379000683008F007E017FD1FE70D831C83612FD9
:1037A0006F70CE010E94621B12951F701061CE01D6
:1037B000612F0E94621B006BCE01602F0E94621B72
:1037C000DF91CF911F910F910895CF93DF93EC017B
:1037D00061E20E94621BCE0160E00E94621BCE018A
:1037E0006FE70E94621BCE0162E20E94621BCE0163
:1037F00060E00E94621BCE0167E00E94621BE989C3
:10380000FA8980819F89892B8083EB89FC8980815B
:10381000988D892B8083E989FA8990818F89809599
:103820008923808340E050E01FC0EF85F8899081B4
:103830008E89809589238083ED85FE8590818D8991
:10384000809589238083EF85F88980819E89892BE3
:1038500080832F5F3F4F2830310539F74F5F5F4F2F
:1038600084E04030580719F020E030E0DECFE989ED
:10387000FA8980819F89892B8083DF91CF91089578
:10388000DC015196ED91FC915297808157969C9165
:103890005797892B80835396ED91FC9154978081A3
:1038A00058969C915897892B80835196ED91FC9165
:1038B0005297908157968C91579780958923808352
:1038C00030E840E050E070E01F96ED91FC91509799
:1038D000908156968C915697809589238083832F6B
:1038E00090E0862397231D96ED91FC911E975596A7
:1038F0002C915597892B21F08081822B808304C0E5
:1039000080812095282320831F96ED91FC9150976C
:10391000808156969C915697892B808336954F5F70
:103920005F4F4830510581F65196ED91FC915297C9
:10393000808157969C91892B808308953F924F9266
:103940005F926F927F928F929F92AF92BF92CF922F
:10395000DF92EF92FF920F931F93DF93CF9300D0EC
:1039600000D0CDB7DEB78C01DC0116968C9116978E
:103970001496FC908130B1F5B7E0FB0EF801F482AB
:10398000862F8052803608F06FE7605285E0689F8E
:103990007001112488E692E0E80EF91ECC24DD24A3
:1039A000F701EC0DFD1DE491C8016E2F0E94401C33
:1039B0000894C11CD11C95E0C916D10489F7FF24D5
:1039C0000CC0D80114968C9114978F5F14968C9329
:1039D000C80160E00E94401CF394F8018781F8164A
:1039E00080F3F3C0D80115968C9085E0689FC001E4
:1039F000112470E6472E7FEF572E480E591EDD2406
:103A000065E6662E6FEF762E680E791ECBC0AD2C64
:103A1000BB24F8018581992787FD90958A0D9B1D10
:103A2000803891050CF0C4C0DD2031F06D2D680D9B
:103A3000C8014F2D0E94C11B53E0AA0CBB1C5A9514
:103A4000E1F73A2C31945C824B82EB81FC81E8599E
:103A5000FD4F9490D8011696FC912F2F30E0C501B0
:103A6000B9010E94E52B81E090E002C0880F991F08
:103A70006A95E2F7E82FC90143E0880F991F4A953C
:103A8000E1F7821B930B432D480FEE2421E0CE2E4D
:103A9000C92030E011C0C110E22A220F4150842F0A
:103AA00090E06F2F70E00E94D12B892B11F4EE0F64
:103AB00005C0222329F03F5F3F1768F3222339F71F
:103AC000D8015196ED91FC915297808157969C9127
:103AD0005797892B80835396ED91FC915497808161
:103AE00058969C915897892B80835196ED91FC9123
:103AF0005297908157968C9180958923808360E0BE
:103B0000EE2DF0E0FA83E98336C030E840E050E083
:103B1000D8011F96ED91FC915097908156968C910B
:103B20005697809589238083832F90E0E981FA81DD
:103B30008E239F231D96ED91FC911E9755962C91F7
:103B4000892B21F08081822B808304C08081209585
:103B500028232083D8011F96ED91FC9150978081F6
:103B600056969C91892B808336954F5F5F4F4830E6
:103B7000510571F66F5FF8018681681730F2018890
:103B8000F289E02D8081D80157969C91892B808302
:103B9000EB81FC813196FC83EB83E615F70509F098
:103BA00054CFD394D80116962C91D21608F42FCF67
:103BB000F8018781F80E85E0289FC0011124F80ED6
:103BC000C801682D4F2D0E94C11B81E090E00F902D
:103BD0000F900F900F90CF91DF911F910F91FF9059
:103BE000EF90DF90CF90BF90AF909F908F907F909D
:103BF0006F905F904F903F900895CF92DF92EF9239
:103C0000FF920F931F93CF93DF936C017B01EB0126
:103C100009900020E9F72197C61BD70B00E010E0C0
:103C20000EC0D601ED91FC91D701A00FB11F0190FC
:103C3000F081E02DC6016C9109950F5F1F4F0C17A5
:103C40001D0778F3CE01DF91CF911F910F91FF9067
:103C5000EF90DF90CF900895CF92DF92EF92FF9296
:103C60000F931F93CF93DF938C01FC011482158275
:103C700081E086838783828561E00E94B520F80118
:103C8000838561E00E94B520F801848561E00E948F
:103C9000B520F8018485282F332727FD309556E677
:103CA000C52E54E0D52EF601E20FF31FE491F0E0AB
:103CB000EE0FFF1F92E5E92E94E0F92EEE0DFF1DA9
:103CC00085919491F801928B818BCAE7D4E02C0FF7
:103CD0003D1FF9018491F801878B8285282F3327B6
:103CE00027FD3095F601E20FF31FE491F0E0EE0FAF
:103CF000FF1FEE0DFF1D85919491F801948B838B2E
:103D00002C0F3D1FF9018491F801808F808561E0BF
:103D10000E94B520F801818561E00E94B520F8017C
:103D20008185282F332727FD3095F601E20FF31FF9
:103D3000E491F0E0EE0FFF1FEE0DFF1D85919491D1
:103D4000F801908B87872C0F3D1FF9018491F801B2
:103D5000868B2085332727FD3095C20ED31EF601B2
:103D60008491E82FF0E0EE0FFF1FEE0DFF1D85910F
:103D70009491F80196878587C20FD31FFE01849125
:103D8000F801858B838561E00E94F42061E070E09A
:103D900080E090E00E942120F801838560E00E948D
:103DA000F4206AE070E080E090E00E942120F801B9
:103DB000838561E00E94F420C8016EEA0E94621BC4
:103DC000C80165ED0E94621BC80160E80E94621B89
:103DD000C80168EA0E94621BC8016FE30E94621B6F
:103DE000C80163ED0E94621BC80160E00E94621B73
:103DF000C80160E40E94621BC8016DE80E94621B5A
:103E0000C80164E10E94621BC80160E20E94621B5B
:103E1000C80160E00E94621BC80161EA0E94621B47
:103E2000C80168EC0E94621BC8016AED0E94621B17
:103E3000C80162E10E94621BC80161E80E94621B26
:103E4000C8016FEC0E94621BC80169ED0E94621BF1
:103E5000C80161EF0E94621BC8016BED0E94621BEA
:103E6000C80160E40E94621BC80164EA0E94621BF0
:103E7000C80166EA0E94621BC8016FEA0E94621BC9
:103E8000DF91CF911F910F91FF90EF90DF90CF9036
:103E90000895823000F5E82FF0E0EE0FFF1FE85B99
:103EA000F94F71836083882319F08130A1F408C031
:103EB000809169008C7F842B80936900E89A089533
:103EC00080916900440F551F440F551F837F842B39
:103ED00080936900E99A0895823080F4882319F06C
:103EE000813021F402C0E89801C0E998E82FF0E0A1
:103EF000EE0FFF1FE85BF94F1182108208951F92A9
:103F00000F920FB60F9211242F933F934F935F930D
:103F10006F937F938F939F93AF93BF93EF93FF9391
:103F20008091480690914906892B29F0E091480636
:103F3000F09149060995FF91EF91BF91AF919F9143
:103F40008F917F916F915F914F913F912F910F9042
:103F50000FBE0F901F9018951F920F920FB60F92E1
:103F600011242F933F934F935F936F937F938F937E
:103F70009F93AF93BF93EF93FF9380914A069091E5
:103F80004B06892B29F0E0914A06F0914B060995E2
:103F9000FF91EF91BF91AF919F918F917F916F9121
:103FA0005F914F913F912F910F900FBE0F901F90F7
:103FB00018951F920F920FB60F9211242F933F93D3
:103FC0008F939F93AF93BF9380915006909151062A
:103FD000A0915206B0915306309154060196A11D4E
:103FE000B11D232F2D5F2D3720F02D570196A11DD8
:103FF000B11D209354068093500690935106A093D0
:104000005206B093530680914C0690914D06A091B4
:104010004E06B0914F060196A11DB11D80934C062E
:1040200090934D06A0934E06B0934F06BF91AF916B
:104030009F918F913F912F910F900FBE0F901F90E6
:1040400018959B01AC017FB7F89480914C06909134
:104050004D06A0914E06B0914F0666B5A89B05C0CF
:104060006F3F19F00196A11DB11D7FBFBA2FA92F77
:10407000982F8827860F911DA11DB11D62E0880F22
:10408000991FAA1FBB1F6A95D1F7BC012DC0FFB7AE
:10409000F89480914C0690914D06A0914E06B091F7
:1040A0004F06E6B5A89B05C0EF3F19F00196A11D8C
:1040B000B11DFFBFBA2FA92F982F88278E0F911DF2
:1040C000A11DB11DE2E0880F991FAA1FBB1FEA9531
:1040D000D1F7861B970B885E9340C8F22150304081
:1040E0004040504068517C4F211531054105510534
:1040F00071F60895789484B5826084BD84B581603A
:1041000084BD85B5826085BD85B5816085BDEEE6DF
:10411000F0E0808181608083E1E8F0E010828081BE
:1041200082608083808181608083E0E8F0E080812C
:1041300081608083E1EBF0E0808184608083E0EB4C
:10414000F0E0808181608083EAE7F0E08081846034
:104150008083808182608083808181608083808190
:10416000806880831092C1000895CF93DF93482F19
:1041700050E0CA0186589B4FFC0134914A595B4F6D
:10418000FA018491882369F190E0880F991FFC015E
:10419000E85BFB4FA591B491FC01EE5AFB4FC59132
:1041A000D491662351F42FB7F8948C91932F909566
:1041B00089238C93888189230BC0623061F42FB7E7
:1041C000F8948C91932F909589238C938881832BDD
:1041D00088832FBF06C09FB7F8948C91832B8C9354
:1041E0009FBFDF91CF910895482F50E0CA018257B9
:1041F0009B4FFC012491CA0186589B4FFC0194916E
:104200004A595B4FFA013491332309F440C0222309
:1042100051F1233071F0243028F42130A1F0223004
:1042200011F514C02630B1F02730C1F02430D9F494
:1042300004C0809180008F7703C0809180008F7DC3
:104240008093800010C084B58F7702C084B58F7DC5
:1042500084BD09C08091B0008F7703C08091B00009
:104260008F7D8093B000E32FF0E0EE0FFF1FEE5A3A
:10427000FB4FA591B4912FB7F894662321F48C914C
:104280009095892302C08C91892B8C932FBF089520
:10429000682F70E0CB0182579B4FFC012491CB012A
:1042A00086589B4FFC0144916A597B4FFB019491C6
:1042B000992319F420E030E03CC0222351F123304F
:1042C00071F0243028F42130A1F0223011F514C00F
:1042D0002630B1F02730C1F02430D9F404C08091E9
:1042E00080008F7703C0809180008F7D8093800055
:1042F00010C084B58F7702C084B58F7D84BD09C09E
:104300008091B0008F7703C08091B0008F7D809343
:10431000B000892F90E0880F991F845A9B4FFC01B1
:10432000A591B4918C9120E030E0842311F021E03C
:1043300030E0C901089508951F920F920FB60F92B1
:1043400011242F933F934F938F939F93EF93FF935A
:104350008091C00082FD1DC04091C6002091D5060D
:104360003091D6062F5F3F4F2F7730708091D70660
:104370009091D8062817390771F0E091D506F09191
:10438000D606EB5AF94F40833093D6062093D506D4
:1043900002C08091C600FF91EF919F918F914F9144
:1043A0003F912F910F900FBE0F901F901895E091A5
:1043B0006907F0916A07E058FF4F81919191208140
:1043C000318180589F4F821B930B60E870E00E9400
:1043D000E52B892B11F00E949B2108951F920F92CB
:1043E0000FB60F9211242F933F938F939F93EF93C8
:1043F000FF932091590730915A0780915B07909164
:104400005C072817390731F48091C1008F7D8093B4
:10441000C10014C0E0915B07F0915C07E752F94FCF
:10442000208180915B0790915C0701968F77907057
:1044300090935C0780935B072093C600FF91EF91F8
:104440009F918F913F912F910F900FBE0F901F90D2
:104450001895AF92BF92DF92EF92FF920F931F9346
:10446000CF93DF93EC017A018B01DD24403081EEA4
:10447000580780E0680780E0780711F0DD24D394C6
:1044800091E0A92EB12CEC89FD89DD2069F0C501F0
:1044900008A002C0880F991F0A94E2F7808360E0A9
:1044A00079E08DE390E005C0108260E874E88EE169
:1044B00090E0A80197010E94F82B21503040404025
:1044C0005040569547953795279580E1203038071D
:1044D00020F0DD2011F0DD24D6CFE889F989308382
:1044E000EA89FB89208319A2EE89FF89408121E0B6
:1044F00030E0C9010C8C02C0880F991F0A94E2F7C2
:10450000482B4083EE89FF894081C9010D8C02C090
:10451000880F991F0A94E2F7482B4083EE89FF89A0
:104520004081C9010E8C02C0880F991F0A94E2F7DE
:10453000482B4083EE89FF8980810F8C02C0220FB7
:10454000331F0A94E2F7209528232083DF91CF912F
:104550001F910F91FF90EF90DF90BF90AF90089563
:10456000DC011C96ED91FC911D97E058FF4F819165
:1045700091912081318180589F4F821B930B60E87D
:1045800070E00E94E52B0895DC011C96ED91FC91F2
:104590001D97E058FF4F20813181E058F040DF0146
:1045A000AE57BF4F8D919C9111972817390719F479
:1045B0002FEF3FEF07C08D919C91E80FF91F80818D
:1045C000282F30E0C9010895DC011C96ED91FC9183
:1045D0001D97E058FF4F20813181E058F040DF0106
:1045E000AE57BF4F8D919C9111972817390719F439
:1045F0002FEF3FEF10C08D919C911197E80FF91F9D
:1046000020818D919C91119701968F7790701196D2
:104610009C938E9330E0C9010895DC0191968C91B2
:104620009197882339F05496ED91FC9155978081AC
:1046300086FFF9CF91961C920895CF93DF93EC01FA
:10464000EE85FF85E058FF4F20813181E058F04032
:104650002F5F3F4F2F773070DF01AE57BF4F8D91E7
:104660009C91119728173907D1F3E058FF4F8081AB
:104670009181E058F040E80FF91F6083EE85FF85D7
:10468000E058FF4F31832083EE89FF89208181E04C
:1046900090E00F8C02C0880F991F0A94E2F7282B34
:1046A000208381E089A3EC89FD89808180648083F7
:1046B00081E090E0DF91CF91089510926007109211
:1046C0005F0788EE93E0A0E0B0E0809361079093ED
:1046D0006207A0936307B093640781E791E090932A
:1046E0005E0780935D0785E596E090936A07809367
:1046F000690789ED96E090936C0780936B0785ECD2
:1047000090E090936E0780936D0784EC90E0909317
:10471000700780936F0780EC90E09093720780930E
:10472000710781EC90E0909374078093730782EC9B
:1047300090E0909376078093750786EC90E09093D5
:1047400078078093770784E08093790783E08093EC
:104750007A0787E080937B0785E080937C0781E080
:1047600080937D0708950895CF93DF930E947A2068
:104770000E94B3230E94CF1AC7EDD1E20E944717CF
:104780002097E1F30E94D721F9CFCF92DF92EF92E9
:10479000FF920F931F93CF93DF937C016B018A01EC
:1047A000C0E0D0E00FC0D6016D916D01D701ED9151
:1047B000FC910190F081E02DC7010995C80FD91F28
:1047C000015010400115110571F7CE01DF91CF9115
:1047D0001F910F91FF90EF90DF90CF900895CF93AE
:1047E000DF93FB01EC01A881B98160817181448173
:1047F00055811296ED91FC9113970995DF91CF9118
:104800000895CF93DF93EC016115710519F420E051
:1048100030E00FC0DB010D900020E9F71197A61BD7
:10482000B70BE881F9810280F381E02DAD01099594
:104830009C01C901DF91CF9108954F925F927F92C1
:104840008F929F92AF92BF92CF92DF92EF92FF92A0
:104850000F931F93DF93CF93CDB7DEB7A1970FB61A
:10486000F894DEBF0FBECDBF2C01742ECB012230D9
:1048700008F42AE019A231E2C32ED12CCC0EDD1EA1
:10488000822E9924AA24BB24672D752FA50194019B
:104890000E94F82B79018A01C801B701A501940192
:1048A0000E94B22B472D461B0894C108D1084A30FC
:1048B00014F4405D01C0495CF6014083E114F10449
:1048C0000105110521F07E2C5F2DC801DDCFC2014D
:1048D000B6010E940124A1960FB6F894DEBF0FBE68
:1048E000CDBFCF91DF911F910F91FF90EF90DF909F
:1048F000CF90BF90AF909F908F907F905F904F90A0
:104900000895DC012115310541F4ED91FC910190F0
:10491000F081E02D642F099508950E941D240895CB
:10492000CF92DF92EF92FF920F931F93CF93DF937B
:10493000EC016A017B012115310541F4E881F9811F
:104940000190F081E02D642F09951FC02A303105B8
:10495000D1F477FF17C0E881F9810190F081E02D53
:104960006DE209958C0144275527BA014C195D0960
:104970006E097F09CE012AE00E941D249801280FAC
:10498000391F04C02AE00E941D249C01C901DF9147
:10499000CF911F910F91FF90EF90DF90CF900895EE
:1049A0000E94012408957F928F929F92AF92BF92AE
:1049B000CF92DF92EF92FF920F931F93CF93DF93EB
:1049C0004C017A018B01722ECB01BA01A80197012B
:1049D0000E94AE2B882321F0C4016BE471E021C05A
:1049E000C0E0D0E057016801E894D7F8C601B501EE
:1049F0002FEF3FEF4FE75FE70E94AE2B882351F484
:104A0000C601B5012FEF3FEF4FE75FE70E94A329F3
:104A1000181614F0C1E0D0E0219739F0C4016FE41A
:104A200071E00E940124EC0193C0C801B7012FEF8F
:104A30003FEF4FE75FE40E94472B181654F0C80180
:104A4000B7012FEF3FEF4FE75FEC0E94A3298823C8
:104A500024F4C40163E571E0E4CFC801B70120E0AC
:104A600030E040E050E00E94A32987FD03C0C0E091
:104A7000D0E00EC0D401ED91FC910190F081E02DC9
:104A8000C4016DE20995EC0117FB109517F910951B
:104A900020E030E040E05FE3DD240BC0CA01B90153
:104AA00020E030E040E251E40E94A7299B01AC01E4
:104AB000D394D71498F3C801B7010E943F295B0132
:104AC0006C010E94142A7B018C01C401B801A7016A
:104AD0002AE030E00E948124C80FD91F772039F0E6
:104AE000C40167E571E00E940124C80FD91FC80105
:104AF000B7010E94402A9B01AC01C601B5010E948A
:104B00003E2924C020E030E040E251E40E944B2BDB
:104B10007B018C010E940F2A5B016C01CC24B7FC45
:104B2000C094DC2CC401B601A5012AE030E00E944B
:104B30009024C80FD91FC601B5010E94422A9B01CB
:104B4000AC01C801B7010E943E297A947720D1F6C2
:104B5000CE01DF91CF911F910F91FF90EF90DF90E9
:104B6000CF90BF90AF909F908F907F9008950E94BC
:104B7000D32408950F931F93CF93DF93EC018B0100
:104B80006F5F7F4F888199810E945D28009711F4A3
:104B900080E005C0998388831B830A8381E0DF91CD
:104BA000CF911F910F910895CF93DF93EC018881EE
:104BB0009981892B29F08A819B818617970760F458
:104BC000CE010E94BA25882341F08C819D81892BDA
:104BD00019F4E881F981108281E0DF91CF91089585
:104BE000EF92FF920F931F93CF93DF93EC017B0122
:104BF0006C817D81E114F104C1F04115510599F0FA
:104C00008A01060F171FB8010E94D425882369F076
:104C1000888199812C813D81820F931FB7010E9469
:104C200086021D830C8381E001C080E0DF91CF917B
:104C30001F910F91FF90EF900895CF93DF93EC01B8
:104C400088819981009711F00E94C52719821882E6
:104C50001D821C821B821A82DF91CF9108950F93CF
:104C60001F93182F092F6115710561F0DB010D905D
:104C70000020E9F71197A61BB70BAD010E94F025A4
:104C8000882321F4812F902F0E941D26812F902FA1
:104C90001F910F9108950F931F93182F092FFB0158
:104CA00060817181448155810E94F025882321F41F
:104CB000812F902F0E941D26812F902F1F910F91E1
:104CC0000895EF92FF920F931F93CF93DF93EC0120
:104CD0007B018A01BA010E94D425882321F4CE01E8
:104CE0000E941D2607C01D830C8388819981B7010E
:104CF0000E948602CE01DF91CF911F910F91FF900C
:104D0000EF900895CF93DF93EC01198218821B82F4
:104D10001A821D821C826115710551F0DB010D9014
:104D20000020E9F71197A61BB70BAD010E94612681
:104D3000DF91CF9108950F931F93182F092F6115BD
:104D4000710559F0DB010D900020E9F71197A61BC2
:104D5000B70BAD010E94612602C00E941D26812F63
:104D6000902F1F910F910895BF92CF92DF92EF92F3
:104D7000FF920F931F93CF93DF93082FB92E6B01F0
:104D80007A01E9012417350710F4EA017901802F2F
:104D90009B2D69E571E00E948226D60114968D91C3
:104DA0009C9115978E159F05D0F08C179D0708F4E0
:104DB000EC01D601ED91FC911197EC0FFD1F1081D4
:104DC00010826D917C916E0D7F1D802F9B2D0E9416
:104DD0009B26D601ED91FC91EC0FFD1F1083802FD7
:104DE0009B2DDF91CF911F910F91FF90EF90DF905E
:104DF000CF90BF900895CF93DF93EC01FB0186170E
:104E0000970761F0608171816115710529F0448116
:104E100055810E94612602C00E941D26CE01DF91AD
:104E2000CF910895FC0111821082138212821582A3
:104E300014820E94FB260895FC01808191810E94CA
:104E4000C5270895FC01808191810E94C52708959E
:104E50000F931F93CF93DF93BC018230910510F421
:104E600062E070E0E0918107F091820740E050E05D
:104E7000A0E0B0E024C08081918186179707D0F030
:104E80008617970771F482819381109729F0139602
:104E90009C938E9312972CC09093820780938107E6
:104EA00027C04115510519F08417950718F48D0195
:104EB000AC01EF01DF01828193819C01F901309700
:104EC000D1F641155105F9F0CA01861B970B8430C4
:104ED000910580F48A819B810115110521F0F8016B
:104EE0009383828304C09093820780938107FE019D
:104EF000329645C0FE01E80FF91F61937193029746
:104F0000998388833CC080917F0790918007892B8B
:104F100041F48091610190916201909380078093A8
:104F20007F0740916301509164014115510541F49F
:104F30004DB75EB780915F0190916001481B590B9E
:104F400020917F073091800724173507B0F4CA01FC
:104F5000821B930B8617970780F0AB014E5F5F4F64
:104F60008417950750F0420F531F509380074093CA
:104F70007F07F9016193719302C0E0E0F0E0CF0197
:104F8000DF91CF911F910F910895CF93DF939C01F3
:104F9000009709F48FC0EC0122971B821A8260915E
:104FA0008107709182076115710581F4888199816B
:104FB000820F931F20917F073091800728173907B0
:104FC00039F5D0938007C0937F0774C0DB0140E0C0
:104FD00050E0AC17BD0708F1BB83AA83FE01219105
:104FE0003191E20FF31FAE17BF0779F48D919C91B9
:104FF0001197280F391F2E5F3F4F39832883129650
:105000008D919C9113979B838A834115510571F46F
:10501000D0938207C09381074DC012968D919C91C9
:105020001397AD01009711F0DC01D3CFDA0113968D
:10503000DC93CE931297FA0121913191E20FF31F85
:10504000CE17DF0769F488819981280F391F2E5FF9
:105050003F4FFA01318320838A819B81938382832E
:10506000E0E0F0E0DB0112968D919C9113970097A0
:1050700019F0BC01FD01F6CFAB014E5F5F4FDB01C4
:105080008D919C91840F951F20917F07309180070F
:105090002817390779F4309729F410928207109273
:1050A000810702C013821282425050405093800701
:1050B00040937F07DF91CF9108956F927F928F92F7
:1050C0009F92AF92BF92CF92DF92EF92FF920F9397
:1050D0001F93CF93DF938C01009729F4CB010E949B
:1050E00028278C01BBC08EEFE82E8FEFF82EE00E44
:1050F000F11E4801860E971E8E149F0408F4ACC062
:10510000D7014D915C91119746175707B8F045307C
:10511000510508F4A3C0CA0104978617970708F43D
:105120009DC042505040461B570BF4014193519390
:105130006D937C93CF010E94C52790C05B01A41A98
:10514000B50A3801640E751EA0918107B0918207DF
:10515000E0E0F0E0CC24DD2447C0A615B705A9F5B2
:10516000CD91DC911197CE0102968A159B0568F1CD
:10517000CE018A199B09029612962C9112971396CA
:105180003C91059758F0F40122833383CA19DB0957
:10519000D183C083D7016D937C9309C04E5F5F4F6D
:1051A0004C0F5D1FF70151834083C901FC01C114FD
:1051B000D10431F0D6011396FC93EE9312974EC0B2
:1051C000F0938207E093810749C08D919C911197DC
:1051D000E817F90708F4FC016D0112968C911297FB
:1051E00013969C919C01D901109709F0B6CF80913C
:1051F0007F079091800786159705E9F4E617F70772
:10520000D0F420916301309164012115310541F4FE
:105210002DB73EB780915F0190916001281B390B3B
:1052200082169306C8F49092800780927F07F70158
:105230007183608313C0CB010E942827EC01009783
:1052400059F0D7014D915C91B8010E947D02C801CF
:105250000E94C5278E0102C000E010E0C801DF9166
:10526000CF911F910F91FF90EF90DF90CF90BF9063
:10527000AF909F908F907F906F9008955058BB276C
:10528000AA270ED0B3C1A4D130F0A9D120F031F4B7
:105290009F3F11F41EF499C10EF4E095E7FB64C141
:1052A000E92FB5D180F3BA17620773078407950712
:1052B00018F071F49EF5E4C10EF4E0950B2EBA2FB0
:1052C000A02D0B01B90190010C01CA01A00111240C
:1052D000FF27591B99F0593F50F4503E68F11A16B8
:1052E000F040A22F232F342F4427585FF3CF469549
:1052F00037952795A795F0405395C9F77EF41F166B
:10530000BA0B620B730B840BBAF09150A1F0FF0F34
:10531000BB1F661F771F881FC2F70EC0BA0F621F20
:10532000731F841F48F4879577956795B795F79510
:105330009E3F08F0B3CF9395880F08F09927EE0FA2
:10534000979587950895ECD008F481E008950CD0E6
:105350004DC145D140F03CD130F021F45F3F19F010
:1053600003C151118EC131C152D198F39923C9F3B0
:105370005523B1F3951B550BBB27AA27621773075B
:10538000840738F09F5F5F4F220F331F441FAA1F0F
:10539000A9F333D00E2E3AF0E0E830D091505040CF
:1053A000E695001CCAF729D0FE2F27D0660F771F7D
:1053B000881FBB1F261737074807AB07B0E809F05F
:1053C000BB0B802DBF01FF2793585F4F2AF09E3FF4
:1053D000510568F0C9C055C15F3FECF3983EDCF35E
:1053E000869577956795B795F7959F5FC9F7880F6D
:1053F000911D9695879597F90895E1E0660F771FBF
:10540000881FBB1F621773078407BA0720F0621B4F
:10541000730B840BBA0BEE1F88F7E095089504D048
:105420006894B1112EC10895FAD088F09F5790F07A
:10543000B92F9927B751A0F0D1F0660F771F881FB9
:10544000991F1AF0BA95C9F712C0B13081F018D17E
:10545000B1E0089515C1672F782F8827B85F39F01C
:10546000B93FCCF3869577956795B395D9F73EF418
:1054700090958095709561957F4F8F4F9F4F0895C0
:10548000E89409C097FB3EF49095809570956195DE
:105490007F4F8F4F9F4F9923A9F0F92F96E9BB2794
:1054A0009395F695879577956795B795F111F8CF10
:1054B000FAF4BB0F11F460FF1BC06F5F7F4F8F4F7B
:1054C0009F4F16C0882311F096E911C0772321F071
:1054D0009EE8872F762F05C0662371F096E8862F09
:1054E00070E060E02AF09A95660F771F881FDAF760
:1054F000880F9695879597F90895ABD080F09F37E0
:1055000040F491110EF0BDC060E070E080E89FEBC8
:10551000089526F41B16611D711D811D2BC045C009
:10552000990F0008550FAA0BE0E8FEEF16161706B4
:10553000E807F907C0F012161306E407F50798F01C
:10554000621B730B840B950B39F40A2661F0232B35
:10555000242B252B21F408950A2609F4A140A695B1
:105560008FEF811D811D089597F99F6780E870E096
:1055700060E00895882371F4772321F09850872BF9
:10558000762F07C0662311F499270DC09051862B02
:1055900070E060E02AF09A95660F771F881FDAF7AF
:1055A000880F9695879597F908959F3F49F09150F8
:1055B00028F4869577956795B7959F5F80389F4FBC
:1055C000880F9695879597F908959FEF80EC089539
:1055D00000240A94161617061806090608950024D2
:1055E0000A9412161306140605060895092E03944C
:1055F000000C11F4882352F0BB0F40F4BF2B11F4C0
:1056000060FF04C06F5F7F4F8F4F9F4F089557FD1E
:105610009058440F551F59F05F3F71F04795880F20
:1056200097FB991F61F09F3F79F0879508951216B7
:1056300013061406551FF2CF4695F1DF08C0161663
:1056400017061806991FF1CF869571056105089414
:105650000895E5DFA0F0BEE7B91788F4BB279F38AF
:1056600060F41616B11D672F782F8827985FF7CF43
:10567000869577956795B11D93959639C8F30895EA
:10568000E894BB2766277727CB0197F9089548DF71
:1056900008F48FEF08950BD0A9CF9ADF28F09FDF91
:1056A00018F0952309F060CF90CF1124EACFAFDF37
:1056B000A0F3959FD1F3950F50E0551F629FF00125
:1056C000729FBB27F00DB11D639FAA27F00DB11D7E
:1056D000AA1F649F6627B00DA11D661F829F222707
:1056E000B00DA11D621F739FB00DA11D621F839F8E
:1056F000A00D611D221F749F3327A00D611D231F64
:10570000849F600D211D822F762F6A2F11249F57B1
:1057100050408AF0E1F088234AF0EE0FFF1FBB1FD4
:10572000661F771F881F91505040A9F79E3F510573
:1057300070F01ACFA6CF5F3FECF3983EDCF386956E
:1057400077956795B795F795E7959F5FC1F7FE2B1E
:10575000880F911D9695879597F90895E1DE880B3E
:10576000990B0895629FD001739FF001829FE00D15
:10577000F11D649FE00DF11D929FF00D839FF00DD0
:10578000749FF00D659FF00D9927729FB00DE11D7C
:10579000F91F639FB00DE11DF91FBD01CF01112459
:1057A0000895AA1BBB1B51E107C0AA1FBB1FA61768
:1057B000B70710F0A61BB70B881F991F5A95A9F7BA
:1057C00080959095BC01CD01089597FB092E072681
:1057D0000AD077FD04D0E5DF06D000201AF47095DA
:1057E00061957F4F0895F6F7909581959F4F0895A5
:1057F000A1E21A2EAA1BBB1BFD010DC0AA1FBB1FD5
:10580000EE1FFF1FA217B307E407F50720F0A21B46
:10581000B30BE40BF50B661F771F881F991F1A94B3
:1058200069F760957095809590959B01AC01BD01DD
:10583000CF010895EE0FFF1F0590F491E02D09941C
:04584000F894FFCF0A
:10584400596F757243616C6C20004D7943616C6CC7
:105854002020200052657065617465722000203E2E
:1058640020004D487A004E54484D45474120362E7D
:10587400350020442D5374617200205350384E5427
:1058840048202620535039414351006E616E00690F
:105894006E66006F7666002E00002C01FA0001800F
:1058A4000083070000000000009E1CC523000000C8
:0E58B400001D23C523B022E422C4220D2300D0
:00000001FF
